:020000040000FA
:040000000EEF00F00F
:04000800B3EF06F05C
:0800180077EF00F0806A896AAD
:10002000070EC16EF30E926E806A816A8A6AF30EC1
:10003000936E816A826A8B6A990E946E600E826EEC
:10004000036A046A056A066A076A026A016A29681D
:100050002A68200E2B6E010E2C6E2D6E006A82B067
:10006000008480B8008281B80080000ECC6EF90E4A
:10007000CB6E040ECA6E0C0EBD6E0C0EBA6EE80E80
:10008000BE6E300EBD12000EBB6E040E806E0C0EE6
:10009000816E796A81B0798081B2798279C078F095
:1000A000C69A400EC76E240EC66EC950C9689E9689
:1000B000D08E9F869D86F29AD59EF194F28CF28E18
:1000C000828C03AA4CEC06F082AEFBD7000082BE05
:1000D000FDD778EC05F061EF00F0F29A810E2E501A
:1000E000D76E2F50D66EF294F28AD58E1200F2B4EB
:1000F00001D01000D58E7D6ED8CF7EF0E0CF7FF09E
:1001000078EC05F02E50D76E2F50D66EF294D58E27
:100110007FC0E0FF7D507EC0D8FF1000183E01D0A8
:10012000172A18501A621200175019621200186A22
:10013000176A1200185006E1175004E11AC018F0AF
:1001400019C017F01806FF0E186212001706176282
:1001500012001200059A23501B62120024501C62E8
:10016000120025501D62120026501E6212000598D2
:100170000596058A120005980596059A23501B647A
:1001800001D01AD01B6001D019D024501C6401D0BA
:1001900013D01C6001D012D025501D6401D00CD0AA
:1001A0001D6001D00BD026501E6401D005D01E600A
:1001B00001D004D0058A12000586120005881200BD
:1001C00037B616D037B40AD037B204D037B001D022
:1001D0001200120037B001D01200120037B204D062
:1001E00037B001D01200120037B001D01200120057
:1001F00037B40DD037B205D037B001D01200058C1E
:10020000120037B002D0058C1200058C120037B2F4
:1002100006D037B002D0058C1200058C120037B022
:1002200002D0058C1200058C120037B617D037B4F7
:100230000BD037B205D037B002D0058C12001200B7
:1002400037B001D01200120037B204D037B001D05D
:100250001200120037B001D01200120037B40CD0D7
:1002600037B204D037B001D01200120037B002D03C
:10027000058C1200058C120037B206D037B002D0C0
:10028000058C1200058C120037B002D0058C1200CC
:10029000058C120037B618D037B40CD037B206D060
:1002A00037B002D0058C1200058C120037B001D097
:1002B0001200120037B204D037B001D01200120081
:1002C00037B001D01200120037B40BD037B204D0CF
:1002D00037B001D01200120037B001D01200058CE7
:1002E000120037B206D037B002D0058C1200058C50
:1002F000120037B002D0058C1200058C120037B600
:1003000019D037B40DD037B206D037B002D0058C33
:100310001200058C120037B002D0058C12001200BA
:1003200037B204D037B001D01200120037B001D07C
:100330001200120037B40AD037B204D037B001D05F
:100340001200120037B001D01200120037B206D0EE
:1003500037B002D0058C1200058C120037B002D0E5
:10036000058C1200058C120037B61AD037B40ED0A7
:1003700037B206D037B002D0058C1200058C1200BF
:1003800037B002D0058C1200058C120037B204D0B1
:1003900037B001D01200120037B001D012001200A5
:1003A00037B40AD037B204D037B001D012001200EF
:1003B00037B001D01200120037B205D037B001D0EB
:1003C0001200058C120037B002D0058C1200058C8B
:1003D000120037B61BD037B40ED037B206D037B0C4
:1003E00002D0058C1200058C120037B002D0058CAB
:1003F0001200058C120037B205D037B002D0058C40
:100400001200120037B001D01200120037B40AD027
:1004100037B204D037B001D01200120037B001D08B
:100420001200120037B204D037B001D0120012000F
:1004300037B002D0058C1200058C120037B61CD0E4
:1004400037B40ED037B206D037B002D0058C1200C8
:10045000058C120037B002D0058C1200058C1200FA
:1004600037B206D037B002D0058C1200058C1200CE
:1004700037B001D01200120037B40AD037B204D01E
:1004800037B001D01200120037B001D012001200B4
:1004900037B204D037B001D01200120037B001D00B
:1004A0001200058C120037B61DD037B40ED037B20B
:1004B00006D037B002D0058C1200058C120037B080
:1004C00002D0058C1200058C120037B206D037B06E
:1004D00002D0058C1200058C120037B002D0058CBA
:1004E0001200120037B40AD037B204D037B001D0AE
:1004F0001200120037B001D01200120037B204D03F
:1005000037B001D01200120037B001D01200120033
:1005100037B61DD037B40DD037B205D037B001D0C3
:100520001200058C120037B002D0058C1200058C29
:10053000120037B206D037B002D0058C1200058CFD
:10054000120037B002D0058C1200058C120037B4AF
:100550000AD037B204D037B001D01200120037B041
:1005600001D01200120037B204D037B001D012000F
:10057000120037B001D01200120037B61CD037B4C9
:100580000CD037B204D037B001D01200120037B00F
:1005900002D0058C1200058C120037B206D037B09D
:1005A00002D0058C1200058C120037B002D0058CE9
:1005B0001200058C120037B40BD037B205D037B01B
:1005C00002D0058C1200120037B001D012001200C8
:1005D00037B204D037B001D01200120037B001D0CA
:1005E0001200120037B61BD037B40BD037B204D08C
:1005F00037B001D01200120037B001D01200058CC4
:10060000120037B206D037B002D0058C1200058C2C
:10061000120037B002D0058C1200058C120037B4DE
:100620000CD037B206D037B002D0058C1200058C42
:10063000120037B001D01200120037B204D037B028
:1006400001D01200120037B001D01200120037B6EC
:100650001AD037B40AD037B204D037B001D0120064
:10066000120037B001D01200120037B206D037B0F6
:1006700002D0058C1200058C120037B002D0058C18
:100680001200058C120037B40DD037B206D037B047
:1006900002D0058C1200058C120037B002D0058CF8
:1006A0001200120037B204D037B001D0120012008D
:1006B00037B001D01200120037B619D037B40AD0C3
:1006C00037B204D037B001D01200120037B001D0D9
:1006D0001200120037B205D037B001D01200058CDD
:1006E000120037B002D0058C1200058C120037B40E
:1006F0000ED037B206D037B002D0058C1200058C70
:10070000120037B002D0058C1200058C120037B2EF
:1007100004D037B001D01200120037B001D012005F
:10072000120037B618D037B40AD037B204D037B079
:1007300001D01200120037B001D01200120037B2FF
:1007400004D037B001D01200120037B002D0058CAF
:100750001200058C120037B40ED037B206D037B075
:1007600002D0058C1200058C120037B002D0058C27
:100770001200058C120037B205D037B002D0058CBC
:100780001200120037B001D01200120037B617D095
:1007900037B40AD037B204D037B001D012001200FB
:1007A00037B001D01200120037B204D037B001D0F8
:1007B0001200120037B001D01200058C120037B4BD
:1007C0000ED037B206D037B002D0058C1200058C9F
:1007D000120037B002D0058C1200058C120037B21F
:1007E00006D037B002D0058C1200058C120037B04D
:1007F00001D01200120037B616D037B40AD037B283
:1008000004D037B001D01200120037B001D012006E
:10081000120037B204D037B001D01200120037B046
:1008200001D01200120037B40ED037B206D037B064
:1008300002D0058C1200058C120037B002D0058C56
:100840001200058C120037B206D037B002D0058CEA
:100850001200058C120037B002D0058C1200120075
:10086000059C000E406207D01EC033F026C037F052
:10087000326A366A20D0010E406209D01DC033F0C2
:1008800025C037F01EC032F026C036F014D0020E5C
:10089000406209D01CC033F024C037F01DC032F0D4
:1008A00025C036F008D01BC033F023C037F01CC081
:1008B00032F024C036F0415012E03B6E06BE05D047
:1008C000334237423B2EFCD70AD033363236D8B0CB
:1008D000338037363636D8B037803B2EF6D70F0EFA
:1008E000331637163350376205D0BBEC00F005B62F
:1008F000058C120033B626D033B412D033B208D0F0
:1009000033B003D0E0EC00F043D015EC01F040D060
:1009100033B003D04AEC01F03BD07FEC01F038D08B
:1009200033B208D033B003D0B4EC01F031D0E9ECED
:1009300001F02ED033B003D01EEC02F029D053ECDE
:1009400002F026D033B412D033B208D033B003D083
:1009500088EC02F01DD0BDEC02F01AD033B003D009
:10096000F2EC02F015D027EC03F012D033B208D02D
:1009700033B003D05CEC03F00BD091EC03F008D063
:1009800033B003D0C6EC03F003D0FBEC03F000D08F
:1009900012002DC03FF01F501B6217D020501C6268
:1009A00014D021501D6211D021501D6205D01B6A48
:1009B0001C6A1D6A1E6A09D01E50225C3F6001D06D
:1009C00004D03F64F4D73F5EF2D73F501E26E86A5A
:1009D0001D221C221B2212002DC03FF0000E1B62A4
:1009E00019D01C6217D01D6215D01D620AD01BC021
:1009F0001FF01CC020F01DC021F01EC022F03F2AB5
:100A000009D03F501E6401D005D01E60F0D71E50A3
:100A10003F5EEDD73F501E5EE86A1D5A1C5A1B5AB6
:100A20001200058423501B620BD024501C6208D096
:100A30001D50FC0B3F6E2550FC0B3F6201D005940E
:100A400012002C502B641200000E0762400E076249
:100A5000800E0762C00E0762120011EC05F005A4BB
:100A600005D02B502D6012002D3612002C502D6415
:100A70001200D8B02D3212002D5005AC02D0075E06
:100A800001D00726000EF86E300EF76E000EF66EDF
:100A90000750060DF4CFF7FFF3CFF6FF0900F5CFAF
:100AA000BEFF0900F5CFBDFF0900F5CFBBFF090070
:100AB000F5CFBAFF0900F5CF80FF1200059E030EA7
:100AC000786012D0020E78600BD0010E786004D0EE
:100AD000020E7962058E1200000E7962058E1200F8
:100AE000030E7962058E1200010E7962058E1200E6
:100AF00004AE28D02A06FF0E2A6224D029C02AF08C
:100B0000AAEC00F005AA03D0049E829C1BD003A48B
:100B100006D0059CBBEC00F005A8058C02D030EC9B
:100B200004F0828C21EC05F03CEC05F005ACC9EC3E
:100B300004F005BCECEC04F0AAEC00F005AA02D02D
:100B4000049E829C796A81B0798081B279827950E1
:100B5000786201D00AD05EEC05F079C078F005AE7D
:100B60008EEC00F005BE9AEC00F01BC010F01CC02B
:100B700011F01DC012F01EC013F017C014F018C001
:100B800015F01200069E030E406E1F5018E01FBEA7
:100B900045EF06F01FBC41EF06F01FBA3DEF06F02F
:100BA0001FB839EF06F01FB635EF06F01FB430EF6F
:100BB00006F01FB22BEF06F01FB026EF06F040063E
:100BC000205018E020BE45EF06F020BC41EF06F0B3
:100BD00020BA3DEF06F020B839EF06F020B635EF29
:100BE00006F020B430EF06F020B22BEF06F020B074
:100BF00026EF06F04006215018E021BE45EF06F032
:100C000021BC41EF06F021BA3DEF06F021B839EFE3
:100C100006F021B635EF06F021B430EF06F021B230
:100C20002BEF06F021B026EF06F04006225033E00D
:100C300022BE45EF06F022BC41EF06F022BA3DEF9E
:100C400006F022B839EF06F049EF06F0030E416EC8
:100C5000068E4BEF06F0020E416E068E4BEF06F04D
:100C6000010E416E068E4BEF06F0000E416E4BEF0B
:100C700006F0010E416E4BEF06F0020E416E4BEF97
:100C800006F0030E416E4BEF06F0040E416E4BEF83
:100C900006F0000E416E1200000E0262120002BC4D
:100CA0003AD002BA2FD002B820D002B601D059D023
:100CB0000AC023F00BC024F00CC025F00DC026F0B4
:100CC0000FC004F004AA08D0049A04A803D00EC0F0
:100CD00029F002D00EC02FF004AC43D029C02AF076
:100CE00003AC3FD06DEC00F03CD00AC01BF00BC051
:100CF0001CF00CC01DF00DC01EF00EC017F00EC091
:100D000018F02FD01BC023F01CC024F01DC025F00C
:100D10001EC026F026D002BAF5D702B812D002B60D
:100D200001D01FD00AC01FF00BC020F00CC021F072
:100D30000DC022F00EC019F00FC01AF0C2EC05F081
:100D400010D00AC02EF00BC02FF00CC02BF00DC03D
:100D50002CF00DC02DF00EC029F00FC003F003A63B
:100D600000D0026A12009D9603BE78EC05F0C950CF
:100D70007A6E0166D2EF06F0070B7C6E0062F4EF2C
:100D800006F07AC07BF07ABA049E7ABC00C010F0FC
:100D900010C0C9FF7ABE02EF07F0060E016E9E96E4
:100DA0009D8611007C500062FDEF06F020EE10F0F1
:100DB0000150D95E7AC0DFFF20EE16F00150D95EF7
:100DC000DFCF7AF0014EEAEF06F07AC0C9FF9E96B7
:100DD0009D861100C9687B50F80B026E03BA4CEC7B
:100DE00006F09E969D861100C9687ABE2EEF07F028
:100DF000060E016E9E969D861100C96801069E969C
:100E00009D861100C7A0FED7C9500A6E1150C96E49
:100E1000C7A0FED7C9500B6E1250C96EC7A0FED72F
:100E2000C9500C6E1350C96EC7A0FED7C9500D6EC5
:100E30001450C96EC7A0FED7C9500E6E1550C96EAA
:100E4000C7A0FED7C9500F6EC9687B50F80B026E61
:100E500003BA4CEC06F09E969D861100C7A0FED703
:100E6000C950C968C7A0FED7C950C968C7A0FED776
:100E7000C950C968C7A0FED7C950C968C7A0FED766
:100E8000C950C968C7A0FED7C950C9689E969D863B
:020E900011004F
:103000003CE80C0000043CE80C6200043CE80CC8FE
:1030100000043CE81C2200043CE81C7C00043CE862
:103020001CD600043CE82C3000043CE82C7600045C
:103030003CE82CC600043CE83C0200043CE83C3E72
:1030400000043CE83C7000043CE83CA200043CE87E
:103050003CBC00043CE83CD400043CE83CE30004F5
:103060003CE83CE800043CE33CE800043CD43CE899
:1030700000043CBC3CE800043CA23CE800043C707A
:103080003CE800043C3E3CE800043C023CE8000410
:103090002CC63CE800042C763CE800042C303CE8CC
:1030A00000041CD63CE800041C7C3CE800041C2204
:1030B0003CE800040CC83CE800040C623CE8000456
:1030C0000C003CE800000C623CE800000CC83CE846
:1030D00000001C223CE800001C7C3CE800001CD6E0
:1030E0003CE800002C303CE800002C763CE8000076
:1030F0002CC63CE800003C023CE800003C3E3CE8BA
:1031000000003C703CE800003CA23CE800003CBCF5
:103110003CE800003CD43CE800003CE33CE8000014
:103120003CE83CE800003CE83CE300003CE83CD4E0
:1031300000003CE83CBC00003CE83CA200003CE84D
:103140003C7000003CE83C3E00003CE83C020000D3
:103150003CE82CC600003CE82C7600003CE82C3013
:1031600000003CE81CD600003CE81C7C00003CE869
:103170001C2200003CE80CC800003CE80C62000087
:103180003CE80C0000083CE80C6200083CE80CC875
:1031900000083CE81C2200083CE81C7C00083CE8D5
:1031A0001CD600083CE82C3000083CE82C760008CF
:1031B0003CE82CC600083CE83C0200083CE83C3EE9
:1031C00000083CE83C7000083CE83CA200083CE8F1
:1031D0003CBC00083CE83CD400083CE83CE3000868
:1031E0003CE83CE800083CE33CE800083CD43CE810
:1031F00000083CBC3CE800083CA23CE800083C70ED
:103200003CE800083C3E3CE800083C023CE8000882
:103210002CC63CE800082C763CE800082C303CE842
:1032200000081CD63CE800081C7C3CE800081C2276
:103230003CE800080CC83CE800080C623CE80008C8
:103240000C003CE8000C0C623CE8000C0CC83CE8AC
:10325000000C1C223CE8000C1C7C3CE8000C1CD63A
:103260003CE8000C2C303CE8000C2C763CE8000CD0
:103270002CC63CE8000C3C023CE8000C3C3E3CE820
:10328000000C3C703CE8000C3CA23CE8000C3CBC50
:103290003CE8000C3CD43CE8000C3CE33CE8000C6F
:1032A0003CE83CE8000C3CE83CE3000C3CE83CD447
:1032B000000C3CE83CBC000C3CE83CA2000C3CE8A8
:1032C0003C70000C3CE83C3E000C3CE83C02000C2E
:1032D0003CE82CC6000C3CE82C76000C3CE82C307A
:1032E000000C3CE81CD6000C3CE81C7C000C3CE8C4
:1032F0001C22000C3CE80CC8000C3CE80C62000CE2
:020000040030CA
:04000000FFFAFEFE07
:00000001FF
